S0120000626F6F746C6F616465722E73726563E7
S21401F0000C9446F80C9463F80C9463F80C9463F82B
S21401F0100C9463F80C9463F80C9463F80C9463F8FE
S21401F0200C9463F80C9463F80C9463F80C9463F8EE
S21401F0300C9463F80C9463F80C9463F80C9463F8DE
S21401F0400C9463F80C9463F80C9463F80C9463F8CE
S21401F0500C9463F80C9463F80C9463F80C9463F8BE
S21401F0600C9463F80C9463F80C9463F80C9463F8AE
S21401F0700C9463F80C9463F80C9463F80C9463F89E
S21401F0800C9463F80C9463F80C9463F811241FBE77
S21401F090CFEFD0E1DEBFCDBF11E0A0E0B1E0E2E806
S21401F0A0FCEF01E00BBF02C007900D92A030B10744
S21401F0B0D9F711E0A0E0B1E001C01D92A030B10780
S21401F0C0E1F70C9438FD0C9400F800000000089558
S21401F0D085B7806285BF88950895D29AD09AD19ACD
S21401F0E0A79AA69AA59AA49AA39AA29AA19AA09A2E
S21401F0F0BB98BA9AB99AD69AD59AB89816988E980D
S21401F1008C98BF988E98D498DC98D39A8B9A8D9ABF
S21401F110DB9ADA9AD89AD99A0895992780FF02C07D
S21401F120DA9801C0DA9A81FF02C0D99801C0D99A4B
S21401F13082FF02C0D8980895D89A08951F93CF9356
S21401F140C7E010E08C2F0E948DF820E030E08FEFB2
S21401F1509FE7000000000000000000000000000023
S21401F1600000019718161906A4F32F5F3F4F2830A9
S21401F17031056CF3C6951F5F133020F38C2F0E9468
S21401F1808DF8CF911F910895CF93C0E087E00E943C
S21401F1908DF820E030E08FEF9FE7000000000000D0
S21401F1A00000000000000000000001971816190674
S21401F1B0A4F32F5F3F4F243031056CF380E00E94AB
S21401F1C08DF820E030E08FEF9FE7000000000000A0
S21401F1D00000000000000000000001971816190644
S21401F1E0A4F32F5F3F4F243031056CF3CF5FC3305C
S21401F1F008F4CCCFCF91089587FF02C0939A01C03F
S21401F2009398880F99270895880F82998160992786
S21401F21008950F931F93CF93082FC0E01C2F802FC4
S21401F2200E94FCF8082F959A8C2F0E9404F9C82F8B
S21401F23095981F5F183098F39927CF911F910F91DA
S21401F2400895EF92FF921F93CF93DF93CDB7DEB76A
S21401F25024970FB6F894DEBF0FBECDBF9C0140E0E9
S21401F26050E088E68983FE013196C901880F892F0F
S21401F270881F990B91958F708183822F880F8B83BE
S21401F2804C839598DB98142F7F01F70181917F01BC
S21401F2900E9409F91F5F1430C0F310E080E00E945D
S21401F2A009F91F5F1430D0F3959A959824960FB6F6
S21401F2B0F894DEBF0FBECDBFDF91CF911F91FF90B7
S21401F2C0EF900895DB9A0895EF92FF920F931F93A4
S21401F2D0CF93DF93EC01E880F9800A811B81D80186
S21401F2E0C7019070A070B0700097A105B10541F4F8
S21401F2F00E9462F9BB27A12F902F8F2D0E9421F922
S21401F3000894E11CF11C011D111DE882F9820A8393
S21401F3101B8380E00E9409F99927DF91CF911F9105
S21401F3200F91FF90EF90089588E190E029E00FB6E5
S21401F330F894A89581BD0FBE21BDFFCFAF92BF92B5
S21401F340CF92DF92EF92FF920F931F93CF93DF93AB
S21401F3505C016A017B01E9014050504F61407040F9
S21401F36018F080E090E023C082EF9FE00E9428FE24
S21401F3708C0184EF9FE00E9428FE0817190779F098
S21401F3808F5F9F4F61F06FEF84EF9FE00E9435FE25
S21401F3906FEF85EF9FE00E9435FEE199FECF9E015B
S21401F3A0B701A601C5010E948FFD81E090E0DF91C3
S21401F3B0CF911F910F91FF90EF90DF90CF90BF906C
S21401F3C0AF9008952F923F924F925F926F927F92E5
S21401F3D08F929F92AF92BF92CF92DF92EF92FF925F
S21401F3E00F931F93CF93DF93CDB7DEB7C450D140B1
S21401F3F00FB6F894DEBF0FBECDBFDC01CB01BA2F2E
S21401F400A92F982F8827FE01EF5FFE4F80839183F7
S21401F410A283B383AA24BB246501150126018601B4
S21401F4207501CE018F5F9E4F0E9464F99927AA2726
S21401F430BB270E2C04C0880F991FAA1FBB1F0A9456
S21401F440D2F7282A392A4A2A5B2A0894A11CB11C19
S21401F450C11CD11C88E090E0A0E0B0E0E80EF91EE7
S21401F4600A1F1B1F94E0A916B104C104D104C8F2F7
S21401F4706624772443016401530184017301CE019C
S21401F4808F5F9E4F0E9464F99927AA27BB270E2CEF
S21401F49004C0880F991FAA1FBB1F0A94D2F7682AB7
S21401F4A0792A8A2A9B2A0894A11CB11CC11CD11C4A
S21401F4B088E090E0A0E0B0E0E80EF91E0A1F1B1FEE
S21401F4C094E0A916B104C104D104C8F26114710410
S21401F4D08104910409F4DCC0AA24BB246501A614A6
S21401F4E0B704C804D90408F04AC0A114B104C10481
S21401F4F0D10421F1D201C1019070A070B0700097C3
S21401F500A105B105D9F41127052DF42CE32C089497
S21401F510E108F108010911098E2D0E948DF8B02F1E
S21401F520AF2D9E2D882720E031E0AC01BD01CE0134
S21401F53001960E949EF9882309F445C0D201C101B3
S21401F5409070A070B0708E010F5F1F4F080F191FCB
S21401F550CE018F5F9E4F0E9464F9D8018C93089468
S21401F560A11CB11CC11CD11C0894211C311C411CBE
S21401F570511CA614B704C804D90408F4B6CF112741
S21401F580052DF42CE32C8FEF90E0A0E0B0E02822CC
S21401F59039224A225B22211431044104510429F400
S21401F5A00894E108F10801091109B02FAF2D9E2D2D
S21401F5B0882720E031E0AC01BD01CE0101960E9412
S21401F5C09EF9882319F480E090E066C0AA24BB2443
S21401F5D065011501260186017501CE018F5F9E4FDB
S21401F5E00E9464F99927AA27BB270E2C04C0880F0E
S21401F5F0991FAA1FBB1F0A94D2F7282A392A4A2A1A
S21401F6005B2A0894A11CB11CC11CD11C88E090E0A7
S21401F610A0E0B0E0E80EF91E0A1F1B1F94E0A91631
S21401F620B104C104D104C8F26624772443016401FD
S21401F630530184017301CE018F5F9E4F0E9464F9CE
S21401F6409927AA27BB270E2C04C0880F991FAA1F2B
S21401F650BB1F0A94D2F7682A792A8A2A9B2A089419
S21401F660A11CB11CC11CD11C88E090E0A0E0B0E058
S21401F670E80EF91E0A1F1B1F94E0A916B104C10467
S21401F680D104C8F2611471048104910409F024CFF5
S21401F6900E9462F981E090E0CC5FDE4F0FB6F894ED
S21401F6A0DEBF0FBECDBFDF91CF911F910F91FF90AF
S21401F6B0EF90DF90CF90BF90AF909F908F907F900C
S21401F6C06F905F904F903F902F9008950F931F93E8
S21401F6D0CF93DF938C010E9428FEEC0121968E5F6A
S21401F6E09F4F70F46C2FC8010E9435FE8D2F99270D
S21401F6F00F5F1F4F682FC8010E9435FEE199FECFAC
S21401F700DF91CF911F910F910895FF920F931F9351
S21401F710F82E8CEE9FE00E9428FE8C0183E0000FFD
S21401F720111F8A95E1F78F2D992787709070082B06
S21401F730192B602F8CEE9FE00E9435FE812F9927B2
S21401F740682F8DEE9FE00E9435FEE199FECF1F9156
S21401F7500F91FF9008958EEF9FE00E9420FE846037
S21401F760682F8EEF9FE00E9435FEE199FECF089547
S21401F770EF92FF920F931F9381EF9FE00E9420FE6E
S21401F7808F3F19F0682F6F5F01C061E0162F80EF81
S21401F7909FE00E9420FE082F153008F459C08F3FC5
S21401F7A061F16FEF80EF9FE00E9435FEE199FECF99
S21401F7B084EF9FE00E9428FEAA27BB278F5F9F4FFA
S21401F7C0A040B04091F48EEF9FE00E9420FE80FDA5
S21401F7D003C00E94C4F8FDCF65E081EF9FE00E9460
S21401F7E035FEE199FECF0E9494F96FEF81EF9FE01D
S21401F7F00E9435FEE199FECF2BC08EEF9FE00E945E
S21401F80020FE80FD25C00E94C4F860E082EF9FE0E4
S21401F8100E9435FE60E083EF9FE00E9435FEE1998D
S21401F820FECF60E070E080E090E00E94E2F988237D
S21401F83021F40E94ABFB0E9494F960E084EF9FE004
S21401F8400E9435FE60E085EF9FE00E9435FE1FEFC7
S21401F850612F81EF9FE00E9435FEE199FECF0F3FB9
S21401F86059F182EF9FE00E9428FE7C0100271127B4
S21401F870C801B7010E94E2F9882321F40E94ABFB7C
S21401F8800E9494F96E2D84EF9FE00E9435FEBB27FF
S21401F890A12F902F8F2D682F85EF9FE00E9435FEB8
S21401F8A06FEF80EF9FE00E9435FE6FEF81EF9FE0E4
S21401F8B00E9435FEE199FECF0E949EF86FEF81EF20
S21401F8C09FE00E9435FEE199FECF0C9400001F9147
S21401F8D00F91FF90EF9008958CEE9FE00E9428FE16
S21401F8E08F5F9F4F09F048C060E080EE9FE00E9466
S21401F8F035FE60E081EE9FE00E9435FE60E084EE1A
S21401F9009FE00E9435FE60E085EE9FE00E9435FE96
S21401F91060E086EE9FE00E9435FE60E087EE9FE0A5
S21401F9200E9435FE60E082EE9FE00E9435FE60E0B8
S21401F93083EE9FE00E9435FE60E088EE9FE00E9425
S21401F94035FE60E089EE9FE00E9435FE60E08AEEBB
S21401F9509FE00E9435FE60E08BEE9FE00E9435FE40
S21401F96060E08CEE9FE00E9435FE60E08DEE9FE049
S21401F9700E9435FEE199FECF04B603FE13C08EEF5A
S21401F9809FE00E9420FE81FD0DC08EEF9FE00E9449
S21401F99020FE82FD07C080EE9FE00E9466FB81E0AC
S21401F9A00E9485FB04B600FE07C084EE9FE00E941D
S21401F9B066FB83E00E9485FB04B602FE07C086EE66
S21401F9C09FE00E9466FB84E00E9485FB04B601FE70
S21401F9D010C004B600FC0DC08EEF9FE00E9420FE12
S21401F9E081FD07C082EE9FE00E9466FB82E00E94D6
S21401F9F085FB8EEF9FE00E9420FE81FF07C08AEE06
S21401FA009FE00E9466FB86E00E9485FB8EEF9FE0EA
S21401FA100E9420FE82FF07C088EE9FE00E9466FBE0
S21401FA2085E00E9485FB84B7877F84BF84B78E7F7D
S21401FA3084BF84B78B7F84BF84B78D7F84BF8EEFEE
S21401FA409FE00E9420FE8D7F682F8EEF9FE00E9430
S21401FA5035FEE199FECF8EEF9FE00E9420FE8B7F60
S21401FA60682F8EEF9FE00E9435FEE199FECF089544
S21401FA70CFEFD0E1DEBFCDBFF89488E190E020E083
S21401FA800FB6F894A89581BD0FBE21BD0E946DF8F2
S21401FA900E946CFC8EE999EF2C0166247724AA2437
S21401FAA0BB24C6EFDFE0450173016201082C04C0E8
S21401FAB0F694E794D794C7940A94D2F7CE010E949D
S21401FAC020FEC81621F06C2DCE010E9435FE08944A
S21401FAD0A11CB11C88E090E0880E991E219694E046
S21401FAE0A916B10408F30E94B8FB80E090E00C94DC
S21401FAF040FE84B195B108950000000008951816DF
S21401FB00190664F400000000000000000000000078
S21401FB1000000000019718161906A4F308958F92A5
S21401FB209F92AF92BF92CF92DF92EF92FF920F9386
S21401FB301F93CF93DF934C017A018B01809168006C
S21401FB4080FDFCCFE199FECF83E0F70100935B00D7
S21401FB5080936800E8958091680086FF0EC08091CA
S21401FB60680080FDFCCFE199FECF81E180936800BB
S21401FB70E8958091680086FDF2CFAA24BB24650132
S21401FB80E901D695C795CE01AA27BB27A816B906BF
S21401FB90CA06DB0648F5B801A7018091680080FD1A
S21401FBA0FCCFE199FECF21E0F501EA0DFB1DE80D42
S21401FBB0F91D808191810C01FA0160935B0020930D
S21401FBC06800E89511240894A11CB11CC11CD11C25
S21401FBD04E5F5F4F6F4F7F4FCE01AA27BB27A816F8
S21401FBE0B906CA06DB06C8F28091680080FDFCCF24
S21401FBF0E199FECF85E0F70100935B0080936800F2
S21401FC00E8958091680086FF0EC08091680080FDAF
S21401FC10FCCFE199FECF81E180936800E895809161
S21401FC20680086FDF2CFDF91CF911F910F91FF9073
S21401FC30EF90DF90CF90BF90AF909F908F900895F8
S21401FC40E199FECF9FBB8EBBE09A99278DB30895AD
S21401FC50E199FECF9FBB8EBBE09A01960DB29FBB8A
S21401FC608EBBE09A802D9DB30895E199FECF9FBB90
S21401FC708EBB6DBB0FB6F894E29AE19A0FBE08955B
S20601FC80FFCFAE
S80401F0000A
